:10000000AA01A628930085100510051083168510F7
:10001000051005100F30860583121308AA182E2824
:100020003A308D00983065203330920042201330F2
:100030008D00883065204220643064204220643086
:10004000642022309200422028302D200C302D20B8
:1000500006302D20AA1413082E282A1492002A1CD8
:100060003C280510033C031C4128412007308D002B
:10007000D0306520031408002A14FE3C0319A1287F
:1000800005142A1C2A1085140F3086051208F03931
:1000900086048510920E2A184228323064200314F8
:1000A000080089008316081483120808A1288F010C
:1000B0008E00FF308E07031C8F07031CA12803301E
:1000C0008D00DF30652059288D01E83E8C008D09B8
:1000D000FC30031C6E288C0703186B288C07640007
:1000E0008D0F6B280C1874288C1C78280000782839
:1000F00008008E00053094000F080D02031D8228B1
:100100000E080C02043003180130031902301405E4
:10011000031DFF30A128103094008D018C01930C39
:10012000920C031C99280E088C070F0803180F0F58
:100130008D078D0C8C0C910C900C940B8F28100853
:10014000A12883130313831264000800831681011E
:100150000F30860085018312FE300220013002201C
:100160002030022020300220413002204330022083
:100170005430022049300220563002204130022003
:100180002030022020300220523002204530022050
:100190004C30022045300220203002202030022046
:1001A000FE300220C0300220203002202030022009
:1001B000203002205B300220393002205D300220E6
:1001C0003D3002204F3002204E3002202F300220DE
:1001D0004F30022046300220463002203721640092
:1001E0003A08003C0319EE2864003C08393C031926
:1001F000FA28EE2864305720FE3002200130022019
:100200002030022020300220493002204E300220CF
:100210004730022052300220453002205330022065
:100220004530022020300220503002204130022090
:100230005330022053300220203002202030022090
:1002400001308F00F4305820F92164003808003C58
:100250000319AC286522792264003808013C03198F
:10026000AC2804308506831605118312AC28BA0128
:10027000FF30BC00703086000F3006059E009F01E5
:100280001E088C001F088D008F010E307920031D81
:100290004E292A30BC000130BA0069291E088C00A2
:1002A0001F088D008F010D307920031D5C2930302F
:1002B000BC000130BA0069291E088C001F088D009F
:1002C0008F010B307920031D69292330BC000130D8
:1002D000BA00B03086000F3006059E009F011E0850
:1002E0008C001F088D008F010E307920031D7D29A1
:1002F0003130BC000130BA0098291E088C001F085C
:100300008D008F010D307920031D8B293230BC0008
:100310000130BA0098291E088C001F088D008F013B
:100320000B307920031D98293330BC000130BA000E
:10033000D03086000F3006059E009F011E088C00FD
:100340001F088D008F010E307920031DAC29343039
:10035000BC000130BA00C7291E088C001F088D00A0
:100360008F010D307920031DBA293530BC000130D2
:10037000BA00C7291E088C001F088D008F010B30A2
:100380007920031DC7293630BC000130BA00E030A7
:1003900086000F3006059E009F011E088C001F0876
:1003A0008D008F010E307920031DDB293730BC0012
:1003B0000130BA00F6291E088C001F088D008F013D
:1003C0000D307920031DE9293830BC000130BA0016
:1003D000F6291E088C001F088D008F010B30792034
:1003E000031DF6293930BC000130BA0032305720E5
:1003F0000800FE300220013002200130B900BA01AD
:1004000037210A30572064003A08003C0319FF29BD
:100410006430572064003C082A3C031D122AB801AE
:100420000800212A64003C08233C031D212A6400A3
:100430000530390203181E2AFF29212A0130B8008D
:1004400008006400053039020318332AFF303907E9
:100450009E00FF300318013E9F001E08303E8400BE
:100460003C088000B90AFE300220013002206400FE
:1004700002303902031C472A0230BB0064003B08EB
:100480003902031C472A2A300220BB0F3E2A64008F
:100490003908053C031D642AFE300220C0300220CA
:1004A0002030022020300220203002202030022084
:1004B0002030022020300220203002205B30022039
:1004C000233002205D300220FF29BB01640004308C
:1004D0003B020318782A3B0851209E009F013B08ED
:1004E000343E84001E0880000A305720BB0F662A65
:1004F0000800BB01640004303B020318A32A3B0838
:10050000303E840000089E00D0301E079E00FF3061
:100510000318013E9F003B08303E84001E08800007
:100520003B08343E840000089E00D0301E079E0029
:10053000FF300318013E9F003B08343E84001E0834
:100540008000BB0F7A2A300892009301E8308E00B9
:1005500003308F008B209E0011089F00310892000D
:10056000930164308E008F018B20A0001108A10040
:100570001E08A0071F080318013EA10732089200B9
:1005800093010A308E008F018B20A2001108A30076
:100590002008A20721080318013EA3073308A20779
:1005A0000318A30A340892009301E8308E00033048
:1005B0008F008B20A4001108A5003508920093013C
:1005C00064308E008F018B20A6001108A70024083C
:1005D000A60725080318013EA707360892009301D5
:1005E0000A308E008F018B20A8001108A900260870
:1005F000A80727080318013EA9073708A80703180A
:0E060000A90A28082202B80008006300052B92
:02400E00FD3F74
:084200003100320033003400EC
:00000001FF
